:100000000C9429070C9470070C9470070C947007DB
:100010000C9470070C9470070C9470070C94700784
:100020000C9470070C9470070C9470260C94442761
:100030000C94E3200C9470070C9470070C947007D8
:100040000C9470070C9470070C9470070C94700754
:100050000C9470070C943A210C9470070C94700760
:100060000C9470070C9470070C9470070C94700734
:100070000C9470070C9470070C9470070C94700724
:100080000C9470070C9470070C9470070C94700714
:100090000C9470070C9470070C9470070C94700704
:1000A0000C9470070C9470070C94700729001E00C4
:1000B0001F0020002100220023002400250026002C
:1000C00027002D002E002A00530054005500560032
:1000D0002B0014001A000800150017001C0018005F
:1000E0000C00120013002F0030004C005F00600075
:1000F00061005700390004001600070009000A00DB
:100100000B000D000E000F003300340031002800FA
:100110005C005D005E005700E10038001D001B0020
:1001200006001900050011001000360037003800E5
:10013000E500520059005A005B005800E000E3005F
:10014000E200000000002C00E700E4005000510035
:100150004F0046004B004E000000000062006300AC
:100160000100010001000100010001000100010087
:100170000100010001000100010001000100010077
:100180000100010001000100010001000100010067
:100190000100010001000100010001000100010057
:1001A0000100010001000100010001000100010047
:1001B0000100010001000100010001000100010037
:1001C0000100010001000100010001000100010027
:1001D0000100010001000100010001000100010017
:1001E0000100010001000100010001000100010007
:1001F00001000100010000000000010001000100F9
:1002000001000100010001000100010000000000E8
:1002100001000100010001000100010001000100D6
:1002200001000100010001000100010001000100C6
:1002300001000100010001000100010001000100B6
:1002400001000100010001000100010001000100A6
:100250000100010001000100010001000100010096
:100260000100010001000100010001000100010086
:100270000100010001000100010001000100010076
:100280000100010001000100010001000100010066
:100290000100010001000100010001000100010056
:1002A0000100010001000100010000000000010048
:1002B0000100010001000100010001000100010036
:1002C0000000000001000100010001000100010028
:1002D0000100010001000100010001000100010016
:1002E0000100010001000100010001000100010006
:1002F00001000100010001000100010001000100F6
:1003000001000100010001000100010001000100E5
:1003100001000100010001000100010001000100D5
:1003200001000100010001000100010001000100C5
:1003300001000100010001000100010001000100B5
:1003400001000100010001000100010001000100A5
:100350000100010001000100010001000100000096
:100360000000010001000100010001000100010086
:100370000100010000000000010001000100010077
:100380000100010001000100010001000100010065
:100390000100010001000100010001000100010055
:1003A0000100010001000100010001000100010045
:1003B0000100010001000100010001000100010035
:1003C0000100010001000100010001000100010025
:1003D0000100010001000100010001000100010015
:1003E0000100010001000100010001000100010005
:1003F00001000100010001000100010001000100F5
:1004000001000100010001000100010001000100E4
:1004100001000000000001000100010001000100D6
:1004200001000100010001000000000001000100C6
:1004300001000100010001000100010001000100B4
:1004400001000100010001000100010001000100A4
:100450000100010001000100010001000100010094
:100460000100010001000100010001000100010084
:100470000100010001000100010001000100010074
:100480000100010001000100010001000100010064
:100490000100010001000100010001000100010054
:1004A0000100010001000100010001000100010044
:1004B0000100010001000100010001000100010034
:1004C0000100010001000000000001000100010026
:1004D0000100010001000100010001000000000016
:1004E0000100010001000100010001000100010004
:1004F00001000100010001000100010001000100F4
:1005000001000100010001000100010001000100E3
:1005100001000100010001000100010001000100D3
:1005200001000100010001000100010001000100C3
:1005300001000100010001000100010001000100B3
:1005400001000100010001000100010001000100A3
:100550000100010001000100010001000100010093
:100560000100010001000100010001000100010083
:100570000100010001000100010000000000010075
:100580000100010001000100010001000100010063
:100590000000000001000100010001000100010055
:1005A0000100010001000100010001000100010043
:1005B0000100010001000100010001000100010033
:1005C0000100010001000100010001000100010023
:1005D0000100010001000100010001000100010013
:1005E0000100010001000100010001000100010003
:1005F00001000100010001000100010001000100F3
:1006000001000100010001000100010001000100E2
:1006100001000100010001000100010001000100D2
:1006200001000100010001000100010001000000C3
:1006300000000100010001000100010001000100B3
:1006400001000100000000000100010001000100A4
:100650000100010001000100010001000100010092
:100660000100010001000100010001000100010082
:100670000100010001000100010001000100010072
:100680000100010001000100010001000100010062
:100690000100010001000100010001000100010052
:1006A0000100010001000100010001000100010042
:1006B0000100010001000100010001000100010032
:1006C0000100010001000100010001000100010022
:1006D0000100010001000100010001000100010012
:1006E0000100000000000100010001000100010004
:1006F00001000100010001000000000001000100F4
:1007000001000100010001000100010001000100E1
:1007100001000100010001000100010001000100D1
:1007200001000100010001000100010001000100C1
:1007300001000100010001000100010001000100B1
:1007400001000100010001000100010001000100A1
:100750000100010001000100010001000100010091
:100760000100010001000100010001000100010081
:100770000100010001000100010001000100010071
:100780000100010001000100010001000100010061
:100790000100010001000000000001000100010053
:1007A0000100010001000100010001000000000043
:1007B0000100010001000100010001000100010031
:1007C0000100010001000100010001000100010021
:1007D0000100010001000100010001000100010011
:1007E0000100010001000100010001000100010001
:1007F00001000100010001000100010001000100F1
:1008000001000100010001000100010001000100E0
:1008100001000100010001000100010001000100D0
:1008200001000100010001000100010001000100C0
:1008300001000100010001000100010001000100B0
:1008400001000100010001000100000000000100A2
:100850000100010001000100010001000100010090
:100860000000000001000100010001000100010082
:100870000100010001000100010001000100010070
:100880000100010001000100010001000100010060
:100890000100010001000100010001000100010050
:1008A0000100010001000100010001000100010040
:1008B0000100010001000100010001000100010030
:1008C0000100010001000100010001000100010020
:1008D0000100010001000100010001000100010010
:1008E0000100010001000100010001000100010000
:1008F00001000100010001000100010001000000F1
:1009000000000100010001000100010001000100E0
:1009100001000100000000000100010001000100D1
:1009200001000100010001000100010001000100BF
:1009300001000100010001000100010001000100AF
:10094000010001000100010001000100010001009F
:10095000010001000100010001000100010001008F
:10096000010001000100010001000100010001007F
:10097000010001000100010001000100010001006F
:10098000010001000100010001000100010001005F
:10099000010001000100010001000100010001004F
:1009A000010001000100010001000100010001003F
:1009B0000100000000000100010001000100010031
:1009C0000100010001000100000000000100010021
:1009D000010001000100010001000100010001000F
:1009E00001000100010001000100010001000100FF
:1009F00001000100010001000100010001000100EF
:100A000001000100010001000100010001000100DE
:100A100001000100010001000100010001000100CE
:100A200001000100010001000100010001000100BE
:100A300001000100010001000100010001000100AE
:100A4000010001000100010001000100010001009E
:100A5000010001000100010001000100010001008E
:100A60000100010001000000000001000100010080
:100A70000100010001000100010001000000000070
:100A8000010001000100010001000100010001005E
:100A9000010001000100010001000100010001004E
:100AA000010001000100010001000100010001003E
:100AB000010001000100010001000100010001002E
:100AC000010001000100010001000100010001001E
:100AD000010001000100010001000100010001000E
:100AE00001000100010001000100010001000100FE
:100AF00001000100010001000100010001000100EE
:100B000001000100010001000100010001000100DD
:100B100001000100010001000100000000000100CF
:100B200001000100010001000100010001000100BD
:100B300000000000010001000100010001000100AF
:100B4000010001000100010001000100010001009D
:100B5000010001000100010001000100010001008D
:100B6000010001000100010001000100010001007D
:100B7000010001000100010001000100010001006D
:100B8000010001000100010001000100010001005D
:100B9000010001000100010001000100010001004D
:100BA000010001000100010001000100010001003D
:100BB000010001000100010001000100010001002D
:100BC000010001000100010001000100010000001E
:100BD000000001000100010001000100010001000E
:100BE0000100010000000000010001000000000001
:100BF000000000002A2B2800000000000000000078
:100C00000000000000000029000000002C1E34201D
:100C1000212224342627252E362D3738271E1F2043
:100C20002122232425263333362E37381F04050688
:100C30000708090A0B0C0D0E0F10111213141516CC
:100C40001718191A1B1C1D2F3130232D35040506CA
:100C50000708090A0B0C0D0E0F10111213141516AC
:100C60001718191A1B1C1D2F3130354C00000000BD
:100C70000000000000000000000000000000000074
:100C80000000000000000000000000000000000064
:100C90007E0F00D4FFFFFFC70000007812036B0037
:100CA0006500790062006F0061007200640000005E
:100CB000160371006D006B006200750069006C0026
:100CC00064006500720000000403090409025B006F
:100CD000030100A0FA090400000103010100092139
:100CE000110100012240000705810308000A0904E0
:100CF000010002030000000921110100012222006D
:100D000007058203200001070503032000010904F1
:100D10000200010300000009211101000122B600B8
:100D20000705840320000A1201000200000008EDFC
:100D3000FE60600100010200010660FF0961A1017F
:100D40000962150026FF00952075088102096315C8
:100D50000026FF00952075089102C005010902A137
:100D60000185020901A100050919012908150025BD
:100D700001950875018102050109300931158125A8
:100D80007F95027508810609381581257F950175C3
:100D9000088106050C0A38021581257F9501750822
:100DA0008106C0C005010980A101850319012AB788
:100DB00000150126B700950175108100C0050C09CA
:100DC00001A101850419012AA002150126A002959E
:100DD0000175108100C005010906A10185050507FF
:100DE00019E029E71500250195087501810205071D
:100DF000190029EF1500250195F0750181020508FC
:100E00001901290595057501910295017503910157
:100E1000C005010906A101050719E029E71500250C
:100E20000195087501810295017508810105071971
:100E30000029FF150026FF009506750881000508AA
:100E40001901290595057501910295017503910117
:100E5000C00011241FBECFEFDAE0DEBFCDBF04B665
:100E600003FE27C08091BD029091BE02A091BF02F7
:100E7000B091C0028730904BA740B04BD1F4109294
:100E8000BD021092BE021092BF021092C00214BEA8
:100E900084B7877F84BF0FB6F894A89580916000CF
:100EA000886180936000109260000FBEE0E0F8E37C
:100EB000099511E0A0E0B1E0EEE6F3E502C005908F
:100EC0000D92AE39B107D9F722E0AEE9B1E001C029
:100ED0001D92AD3BB207E1F70E94F0170C947A29FE
:100EE0000C94000090E080E008950895089581E05A
:100EF000089580FF07C0539A5B9881FF05C0559AFB
:100F00005D9808955398F8CF5598FACF81E00895E9
:100F10000C94770708950C948A071F93CF93DF935F
:100F200000D000D00F92CDB7DEB749835A836B83D0
:100F30003091A00189819A8131111DC06623B9F0D9
:100F40002223A9F00E94E90D182F682F89819A8128
:100F50000E94950D69817A81812F0F900F900F90DB
:100F60000F900F90DF91CF911F910C94961C0E94CF
:100F7000C10D182FEFCF0E94E90D69817A81EDCF65
:100F8000FC01262F408151816281738184810C9400
:100F90008D0781E00895CF93DF93EC0160E00E941C
:100FA000C007BE01DF91CF910C948B07E1E0F0E028
:100FB000DF0102C0AA0FBB1F6A95E2F7BD01DF0186
:100FC00002C0AA0FBB1F4A95E2F76A2B01C0EE0FC1
:100FD0002A95EAF7962F9823961302C08E2B089530
:100FE000E0958E230895242F462F682F8091C50108
:100FF0000E94D6070C94520D0E945C160E94430971
:101000000C9476160C94781608950E94EA0C0E94AF
:1010100004082FEF84E39CE0215080409040E1F7EA
:1010200000C000000C945E210F931F93CF93DF93B9
:101030008C0161E00E94C007EC01B8010E94DD1A3A
:101040008823D9F1B801CE010E9488078823A9F12D
:10105000B801CE010E94CD1D882379F1B801CE01DF
:101060000E941F1E882349F1B801CE010E94421F31
:10107000882319F1F8018281882361F0CA35FDE5E2
:10108000DF0721F170F4C115ECE5DE07A1F0CE3DDC
:10109000DC45C9F0C801DF91CF911F910F910C94ED
:1010A0008607CB358DE5D807A1F0CC35DD4591F726
:1010B0000E94B111EFCF0E94050880E0DF91CF912F
:1010C0001F910F9108950E942713F7CF0E94BA1124
:1010D000E1CF0E94BD11DECFDF92EF92FF920F931E
:1010E0001F93CF93DF93E82FF0E0E451F44FD490B7
:1010F000282F26952695269530E0F901E457F34FE1
:101100000491877010E0082E02C0159507950A9487
:10111000E2F701701127F901E458F34FE490F12C44
:10112000082E02C0F594E7940A94E2F791E0E922D0
:10113000FF24F901E459F34FC491D0E002C0D595E2
:10114000C7958A95E2F7C170DD270115110519F0E1
:1011500081EE0E948F09E114F10419F086EE0E94DD
:101160008F098D2D0E948E0AEF2819F086EE0E94BD
:10117000210A012B19F081EE0E94210ACD2B51F09A
:101180008CE2DF91CF911F910F91FF90EF90DF9054
:101190000C948E0ADF91CF911F910F91FF90EF90E9
:1011A000DF900895EF92FF920F931F93CF93DF93F9
:1011B000EC01162F0AE08881882309F454C081309D
:1011C00009F04EC08981813099F47E0122E0E20E5F
:1011D000F11C8A810E948E0AE7012196812F81509D
:1011E00050F3EFE9FFE03197F1F700C00000F7CFCF
:1011F000823041F47E0182E0E80EF11C8A810E9477
:101200008F09EACF833041F47E01E2E0EE0EF11C5B
:101210008A810E94210AE0CF843011F02196DDCF2F
:101220002A81229690E080E0AE014F5F5F4F20530D
:10123000330B2A30310548F0019778F2EFE9FFE0EF
:101240003197F1F700C00000F7CF089FB001099F68
:10125000700D1124C901860F971F2981EA01E4CF7F
:101260000E946C08BACFDF91CF911F910F91FF9030
:10127000EF90089560E00C94D2080C94790781E017
:1012800008950C943F090895CF93C82F0E943D09FB
:101290008C2FCF910C944109CF93DF93CDB7DEB75C
:1012A0002B970FB6F894DEBF0FBECDBF4F83588784
:1012B00069877A878B8761110E94E0111E821D82E7
:1012C00085E0FE013796DE01119601900D928A9518
:1012D000E1F78C819D81892B89F449815A816B8149
:1012E0007C818D819E810E94E0102B960FB6F89430
:1012F000DEBF0FBECDBFDF91CF91089589819A8166
:1013000089238F3F51F3CE0101960E94C9078111B5
:10131000E4CFEBCFFC01808191810C94160ECF932A
:10132000C82F882309F48BC08238C1F40E94711F32
:1013300081FD85C089E30E947A110E9410122FEF6F
:1013400081EE94E0215080409040E1F700C0000021
:1013500089E30E948111CF910C9410128338A1F47B
:101360000E94711F80FD6BC083E50E947A110E946C
:1013700010122FEF81EE94E0215080409040E1F771
:1013800000C0000083E5E5CF8438A1F40E94711FFE
:1013900082FD55C087E40E947A110E9410122FEF3F
:1013A00081EE94E0215080409040E1F700C00000C1
:1013B00087E4CFCF8CEF8C0F813A90F46C2F809123
:1013C0000001909101010E94E51F882329F08C2FD4
:1013D0000E9481110E9410128C2F0E947A11BBCFA3
:1013E00080E28C0F883048F4C77081E001C0880F1C
:1013F000CA95EAF70E94C311AECFEBE5EC0FE330DC
:1014000040F4F0E0ED5BFE4F808190E0CF910C94D2
:10141000A51FE8E5EC0FE73150F4F0E0EE0FFF1FF9
:10142000EB5EFE4F80819181CF910C94BB1FC03F3A
:1014300030F08C2F0E947E18CF910C945119CF91CF
:101440000895882309F452C0823871F40E94711FF4
:1014500081FF4CC089E30E947A110E94101289E337
:101460000E9481110C941012833859F40E94711F4C
:1014700080FF3CC083E50E947A110E94101283E530
:10148000EFCF843859F40E94711F82FF2FC087E488
:101490000E947A110E94101287E4E2CF9CEF980F0D
:1014A000913AF0F290E2980F983050F4877091E002
:1014B00001C0990F8A95EAF7892F0E94C911D2CFEE
:1014C0009BE5980F933020F490E080E00C94A51FEA
:1014D00098E5980F973120F490E080E00C94BB1FC2
:1014E000803F20F00E94D8180C94511908951F9342
:1014F000CF93DF93182FEB010E948F09209731F4CF
:10150000812FDF91CF911F910C94210A8FE99FE0E9
:101510000197F1F700C000002197F0CF70E060E084
:10152000893311F460E570E00C94770A882321F088
:101530000E94C3110C9410120895882321F00E9478
:10154000C9110C9410120895BF92CF92DF92EF92BE
:10155000FF920F931F93CF93DF936C01D62FC72F6A
:10156000FC011281058102950F700E949811E82EEE
:101570008823A1F0E12E112389F08C2F807F803405
:1015800029F080E28D0FE12C883040F082E00E944B
:1015900061120E94981191E0E82EE926BC2EB294C7
:1015A0009FE0B922EB2DF0E0E458F64D0C940A29A7
:1015B0000C2F0F70C07F11F00295007F1123A9F04E
:1015C000002359F080E28D0F883010F0D11109C04E
:1015D000802F0E94C3110E9410128D2F0E948F092C
:1015E00014C0802F0E94D311F6CF8D2F0E94210AA4
:1015F000002359F080E28D0F883010F0D1112CC0FB
:10160000802F0E94C9110E9410122B2D2850330BDD
:101610002430310520F40E94711F0E944409EE20FD
:1016200009F479C10E94941180FD75C1F6011282FE
:101630000E948E110E94630DC6010E94AC0C0E9494
:101640008E11DF91CF911F910F91FF90EF90DF905E
:10165000CF90BF900C946E0D802F0E94D911D3CFE4
:10166000FC2FFF70FF2EC07FC03219F0F29480EF84
:10167000F822DD2369F0D13049F1112391F10023E3
:1016800051F1F601858180FFA8CF8F70858323C03B
:10169000112381F0011106C00E94F3118F290E94CD
:1016A000960AB3CF0130C1F70E94F3118F290E942F
:1016B000F911ABCF011106C00E9406128F2D0E94B6
:1016C0009D0AA3CF013009F4A0CFF6CF112329F052
:1016D000063008F09ACF8F2DE2CF053008F095CF75
:1016E000EDCF002359F3D93349F4FFEF27EE33E070
:1016F000F15020403040E1F700C000008D2F0E94E3
:10170000210A83CF8C2F86958695837069F081306E
:1017100009F07BCF8D2F9C2F9370111102C090E0A8
:1017200080E00E94BB1F71CF8D2F9C2F93701111F1
:1017300002C090E080E00E94A51F67CF8D2F11238B
:1017400029F00E947E180E9451195FCF0E94D8187C
:10175000FACF8C2F837079F5111157CF4D2F429509
:1017600046954770440F440F8D2F8F70042E01C093
:10177000880F0A94EAF72D2F2071D4FF07C02FE0BD
:1017800030E001C0220F4A95EAF72095C695C6952C
:10179000C370822BC23049F058F4C13019F00E9456
:1017A000440D33CF0E943F0D30CF0E94490D2DCF05
:1017B0000E943D0D2ACF8695112311F08C2F817048
:1017C000882309F422CF4D2F429546954770440F48
:1017D000440F8D2F8F70042E01C0880F0A94EAF7F2
:1017E0002D2F2071D4FF07C02FE030E001C0220F61
:1017F0004A95EAF72095C695C695C370822BC230EC
:1018000049F058F4C13019F00E948A0DFECE0E94B2
:10181000850DFBCE0E948F0DF8CE0E94520DF5CEA5
:10182000CF70112329F08C2F0E94630D8D2F37CF9D
:101830008D2F0E949D0A8C2F0E946E0DE6CED23F06
:1018400089F160F4D03FC9F0D13F29F1112309F4A7
:1018500042C00111C2CE8C2F8F7121C0D33F39F10C
:10186000D43FA1F7112369F1CF718C2F0E94630D32
:1018700063E08C2F0E944612C8CE112341F0053040
:1018800008F0C3CE8C2F8F710E947A0DBECE063029
:1018900008F0BBCEF7CF8C2F8F71112369F20E9415
:1018A000630DB3CE8C2F8F711123C9F3C5CF1123D4
:1018B00029F08C2F8F710E945B0DA7CE0E94580DCE
:1018C000A4CE81E00E946112023008F49ECE82E034
:1018D0000E9461129ACE002359F0D93309F00ECF3D
:1018E0008FEF97EEE3E081509040E040E1F704CFC6
:1018F0008C2F8F71A1CF4C2F4F706D2FC6010E947E
:1019000072070E94440E81CE4C2F4F706D2FC6017E
:101910000E9445147ACEDF91CF911F910F91FF90D5
:10192000EF90DF90CF90BF9008950F931F93CF93C8
:10193000DF93EC01688179818A810E94200E8C01FD
:101940000E94940D0E943C0DB801CE01DF91CF9111
:101950001F910F910C94A40ACF93DF93EC018B811C
:101960009C81892B29F08881998189238F3F59F4A3
:10197000DF91CF910895CE010E94950CCE01DF91A9
:10198000CF910C94CB07CE010E9414088111F3CFA4
:101990000E949811882361F38A81882349F382E0A9
:1019A000DF91CF910C94611290E080E00E94A51F1E
:1019B00090E080E00E94BB1F0E94E0110E94F011A5
:1019C0000E9410120E94781A0C9451190E948811DA
:1019D0000C94D40C0E94D0110C94E60CE92FE295E3
:1019E000EF70E250EE3070F4F0E0E457F64D0C94F6
:1019F0000A29803F19F020F4883E20F481E0089500
:101A0000843FE1F380E00895883EC0F3813FD1F741
:101A1000F5CF93FB882780F90895FC01808191819F
:101A20000E94160E0C94EE0CCF93DF9300D000D0E2
:101A30000F92CDB7DEB70F900F900F900F900F90D1
:101A4000DF91CF910895CF93DF9300D000D000D0E5
:101A5000CDB7DEB726960FB6F894DEBF0FBECDBF6A
:101A6000DF91CF91089508950C94330D0E94340DA9
:101A70008093C6010C94D40C08950C94360D90916B
:101A8000C601892B0C94360D9091C60189230C94C4
:101A9000360D9091C60189270C94360D0C94330DA8
:101AA0000C944E0D0E94500D8093C5010C94D40CE3
:101AB00080E00C94520D91E001C0990F8A95EAF7ED
:101AC000892F0C94520D21E030E001C0220F8A953D
:101AD000EAF78091C501822B0C94520D21E030E091
:101AE00001C0220F8A95EAF720958091C5018223D3
:101AF0000C94520D21E030E001C0220F8A95EAF7E4
:101B00008091C50182270C94520D9091C501892BBB
:101B10000C94520D9091C50189230C94520D909113
:101B2000C50189270C94520D089522E1929F800DE2
:101B30001124982F977041E001C0440F9A95EAF75D
:101B400086958695869593E0899FF0011124EF553F
:101B5000FE4F90E080E070E05191DF0111979B0112
:101B6000082E02C0369527950A94E2F72170219538
:101B70002527242325272C9301968330910561F78F
:101B8000089522E1929F800D1124982F97708695D9
:101B90008695869523E0829FF0011124EF55FE4F34
:101BA00050E040E080E0219130E0092E02C03695FF
:101BB00027950A94E2F721703327042E01C0220FE3
:101BC0000A94EAF7822B4F5F5F4F4330510559F774
:101BD0000895CF92DF92FF920F931F93CF93DF93DD
:101BE0006C010091C5018091C601082BC7E0D0E0CF
:101BF00010E0FC2EC8010C2E02C0959587950A9422
:101C0000E2F780FD0CC02197A0F7F12C8F2DDF911A
:101C1000CF911F910F91FF90DF90CF900895B60163
:101C20008C2F0E946115019771F3F0CFCF93DF9352
:101C3000EC010E94E90DBE01DF91CF910C9461157A
:101C40001F93CF93DF93EB019091A001992331F083
:101C5000CB01DF91CF911F910C94160E882379F060
:101C6000CB010E94E90D182F682FCE010E94950D1F
:101C7000BE01812FDF91CF911F910C946115CB0193
:101C80000E94C10D182FF4CFEF92FF920F931F9374
:101C9000CF93DF938C01892B81F0F12CEE24E39418
:101CA000E8012196F8018491843770F4843008F0BB
:101CB0005FC08130B1F08230A1F1DF91CF911F91EF
:101CC0000F91FF90EF900895853709F44CC008F408
:101CD0003DC09CE7980F903780F78F770E94210ACC
:101CE00049C00E5F1F4FFE01849190E2980F98301B
:101CF00060F48770FE2D01C0FF0F8A95EAF78F2FE1
:101D00000E94E3110E94101202C00E948F098F2DC1
:101D1000815030F2EFE9FFE03197F1F700C00000A9
:101D2000F7CF0E5F1F4FFE01849190E2980F98301D
:101D300050F48770FE2D01C0FF0F8A95EAF78F2FB0
:101D40000E94E911DFCF0E94210AE1CF0E5F1F4FF1
:101D5000FE01C491C150D8F28FE99FE00197F1F7DD
:101D600000C00000F7CF0E5F1F4FFE01F490CFCFF1
:101D70000E948F098E01CBCF1F93CF93DF93C09129
:101D8000C70116E08091C8018C1304C0DF91CF9188
:101D90001F910895D0E01C9FF0011D9FF00D1124AC
:101DA000E753FE4F40815181628173818481958127
:101DB0000E94230D2196C770E5CF4091F901509103
:101DC000FA016091FB017091FC018091FD019091FD
:101DD000FE010C94230D1F93CF93DF938091FE019E
:101DE000807FA9F48091FB01882389F08091C7014D
:101DF000C091C8016091F9017091FA01A091FC01B4
:101E0000B091FD01D62FD72316E0C81304C0DF918F
:101E1000CF911F91089590E0109711F0DF3F19F4D2
:101E200001968770F2CF189F9001199F300D1124F1
:101E3000F901E753FE4F41814713F2CF408146132A
:101E4000EFCF42814111ECCF438154814A1B5B0BA0
:101E5000483C510528F78091FE018F708061809386
:101E6000FE01F901E253FE4F80818F708061808313
:101E700089EF91E00E94AC0CDF91CF911F910C94FF
:101E8000BC0EAF92BF92CF92DF92EF92FF920F9370
:101E90001F93CF93DF93CDB7DEB761970FB6F8945A
:101EA000DEBF0FBECDBF8C0185E0F801DE011D96BF
:101EB00001900D928A95E1F7F801E28089EFC82E32
:101EC00081E0D82E6091FC017091FD0161157105D2
:101ED00009F45AC19091F9012091FA01892F8223C6
:101EE0008F3F09F451C140815181A380B480F090AB
:101EF000FB01F501E61BF70BFF2009F4F6C080910A
:101F0000FE01382F307FE83CF10508F0AFC03111F9
:101F100079C0FE2C251323C0941321C0E1101FC0EB
:101F20008F7080618093FE010E94DD0EC6010E94C9
:101F3000AC0C8091FE01F80185838F2D61960FB660
:101F4000F894DEBF0FBECDBFDF91CF911F910F91EF
:101F5000FF90EF90DF90CF90BF90AF900895AB28A7
:101F600029F0842F85238F3F09F027C180E0F82FC7
:101F7000F170DF2E80FF3CC08091C7012091C80125
:101F800036E0821315C04D875E878D859E850E9441
:101F9000160E292F22952F702230F0F0243018F5DC
:101FA0009F70F1F0F8019581907FD1F4D12C1EC083
:101FB00090E0389FF001399FF00D1124E753FE4F58
:101FC0006181651306C06081641303C06281E612FB
:101FD0000FC001968770D5CF9F7011F0882331F321
:101FE000805E883018F3C8010E94AC0CFD2CA5CF90
:101FF000EE2009F4A2CF8091FE0181608093FE0162
:10200000F12C9BCF251306C0941304C0F801EE20D9
:1020100009F487C0C8010E940D0D882319F1EE2034
:1020200009F18091FE01803270F02091F901309128
:10203000FA0138872F831986BB86AA868C87CE0142
:1020400007960E94AC0C86E0F801A9EFB1E0019080
:102050000D928A95E1F70E94EB0E0E94DD0EFF249F
:10206000F3946BCFC8010E94AC0CF9CF311113C0AF
:102070007A2DB98AA88A6E2D89890E94140D89EF5C
:1020800091E00E94AC0C86E0F60111928A95E9F786
:102090000E94DD0EB5CF25130FC094130DC0E110C3
:1020A0000BC0F8018583C8010E94AC0C86E0F601E4
:1020B00011928A95E9F741CFC8010E940D0D88233E
:1020C00089F2EE2079F28091FE01803208F4BBCFD4
:1020D0002091F9013091FA013A8329831B82BD8254
:1020E000AC828E83CE010196ACCFE83CF10508F0BE
:1020F0003EC0FE2CEE2009F4B5CF25132AC0941360
:1021000028C08091FE0180FD1BC0982F907FC1F0F8
:10211000F8018583903F31F0982F907F905F8F700A
:10212000892B8583C8010E94AC0C86E0F801A9EFD9
:10213000B1E001900D928A95E1F70E94DD0EFDCE8F
:1021400086E0F801A9EFB1E001900D928A95E1F7E0
:10215000F4CEC8010E940D0D811175CF8091FE0152
:1021600081608093FE01C8010E94AC0CE6CE7A2DFE
:10217000B98AA88A6E2D89890E94140D86E0F6011D
:1021800011928A95E9F7D9CFEE2009F46BCFC801F7
:102190000E940D0DF82E882309F464CF86E0F80123
:1021A000A9EFB1E001900D928A95E1F789EF91E0F6
:1021B0000E948A090E94EB0EC0CF81E08E25D7CE07
:1021C0001F93CF93DF93CDB7DEB72C970FB6F8945C
:1021D000DEBF0FBECDBF4F83588769877A878B8755
:1021E0009C87CE0107960E94410F882369F08A855B
:1021F0009B85892B39F04F815885842F85238F3F0C
:1022000009F071C016E05FC086E0FE013796DE017E
:10221000119601900D928A95E1F78A859B85892B0D
:1022200089F38F81988589238F3F61F32091C801BD
:1022300030E0C9010196877099274091C70148177E
:10224000190671F40E94EA0C1092C8011092C7019D
:1022500086E0E9EFF1E0DF011D928A95E9F7D2CF40
:1022600096E0929FD001939FB00D1124A753BE4FCB
:10227000FE01319601900D929A95E1F78093C80185
:102280000E94BC0EBFCF819FC001112487539E4F77
:102290000E94410F8823E9F0E091C7011E9FF001E1
:1022A0001124E753FE4F4081518162817381848103
:1022B00095810E94230D8091C70190E0019687705F
:1022C00099278093C7018091C7019091C801891314
:1022D000DACF2C960FB6F894DEBF0FBECDBFDF91DC
:1022E000CF911F91089569857A858B859C850E9481
:1022F000230D88CF682F80910001909101010C94EB
:102300006520682F80910001909101010C9470204C
:1023100080910001909101010C947B208091FF013C
:1023200085958595859508958091FF01877008951D
:102330009091FF01977081E009F480E008959091F9
:10234000830292FB222720F9281751F080FB92F993
:102350009093830280918202909183020C94A41244
:1023600008958091830282FB882780F991E0892774
:102370000C949F1181E00C949F1180E00C949F11AC
:1023800080912302089590912302892B8093230248
:1023900008958095909123029823909323020895A5
:1023A00010922302089590912202892B8093220299
:1023B0000895809590912202982390932202089587
:1023C00010922202089590912102892B809321027C
:1023D0000895809590912102982390932102089569
:1023E00010922102089580910002089508950C949E
:1023F000F6119091830292FD08C090910002981707
:1024000021F0809300020C94F7110895809100024E
:10241000882329F01092000280E00C94F7110895AF
:10242000E0910001F0910101809123028083E0910D
:102430000001F0910101808190912202892B80831B
:10244000E0910001F0910101808190912102892B9E
:10245000808390910002992381F0E0910001F09136
:1024600001018081892B808380910001909101017D
:102470000E94D11F81110E9406128091000190914B
:1024800001010C947D1F08950C94431290918302D6
:1024900092FD10C098E0899F90011124622B6093F7
:1024A000FF010E94630D8091FF01859585958595BB
:1024B0000C9444120C94630D1092FF0180E00C9474
:1024C00044129091FF01809589238093FF01282F6A
:1024D000277039F4282F082E000C330B921713069F
:1024E00021F49091830292FF07C08595859585958B
:1024F0000E946E0D0C945C1208956FEF7FEF90E0D8
:1025000080E00C94642990E080E00E944029893E9C
:102510009E4F11F40C94861A80E0089582E090E0BA
:102520000C94382983E090E00C943829CF9384E010
:1025300090E00E943829C82F82E290E00E9438295A
:10254000982F8C2FCF910895CF93C92F682F84E0B7
:1025500090E00E9446296C2F82E290E0CF910C948B
:102560004629AB01BC018FE090E00C945829AB01E7
:10257000BC0183E190E00C94582960E070E0CB014D
:102580000C94B71260E070E0CB010E94B1120C9481
:10259000BD1269EE7EEF90E080E00E94642960E069
:1025A00082E090E00E94462960E083E090E00E9493
:1025B00046291092C60160E084E090E00E9446291E
:1025C00060E082E290E00E94462960E085E090E0D1
:1025D0000E94462960E086E090E00E9446296FEF65
:1025E00087E090E00E94462940E050E0BA0188E090
:1025F00090E00E94582960E08DE090E00E9446291A
:1026000040E050E0BA0188E190E00E94582960E083
:1026100087E190E00E94462940E050E0BA018CE159
:1026200090E00E94582970E060E080E290E00E9413
:10263000642940E050E0BA0188E190E00E94582906
:1026400080E00E949F1A0E94C51A0C94C2120C943A
:10265000C912682F8EE090E00C9446290E941F2139
:1026600060933D0270933E0280933F02909340023C
:102670006093390270933A0280933B0290933C023C
:10268000089585B7806885BF85B7806885BF089540
:10269000089508950C94481308950C944C130E94C7
:1026A00041138FE396E10E9482210E9449130C940A
:1026B0004A1381E008950C945913089508950E94D7
:1026C0005D130C945E130E940A210E94D41A0E948A
:1026D00052170C944D134F925F926F927F928F928C
:1026E0009F92AF92BF92CF92DF92EF92FF920F93A1
:1026F0001F93CF93DF93CDB7DEB72A970FB6F89429
:10270000DEBF0FBECDBF0E94691781110E942E133C
:1027100055E2A52E52E0B52E10E000E0802E802F6D
:102720000E947A162B013C01F501C190D190E190F5
:10273000F1905F01C414D504E604F70409F477C0EE
:102740008091410281FD0E948516D701C601842532
:102750009525A625B725912CC12CD12C7601C394A3
:10276000AC01BD014C215D216E217F21452B462B03
:10277000472B09F454C00E945B138823C9F09E8242
:102780008F824C205D206E207F2081E045284628E6
:10279000472809F480E088870E9413218160782F00
:1027A0009A8789874E815F8168858A850E944C0956
:1027B000000F111F000F111FF801EB5DFD4F80810D
:1027C0009181A281B3818C259D25AE25BF25808373
:1027D0009183A283B3830E946C190E94711F909110
:1027E00024028917D9F10E94711F809324022A962E
:1027F0000FB6F894DEBF0FBECDBFDF91CF911F9112
:102800000F91FF90EF90DF90CF90BF90AF909F908F
:102810008F907F906F905F904F900C9444099394A9
:10282000CC0CDD1CEE1CFF1CF2E19F1299CF0F5F58
:102830001F4F0530110509F071CF8FEF89838A830F
:102840001B820E9413218160782F9D838C83498194
:102850005A816B818D810E944C09BDCF2A960FB69B
:10286000F894DEBF0FBECDBFDF91CF911F910F91C6
:10287000FF90EF90DF90CF90BF90AF909F908F90A0
:102880007F906F905F904F9008950895FC01EE0F38
:10289000FF1FE456F34F859194910895CF93DF93F2
:1028A0000E946515EC01811520E5920708F042C0F1
:1028B000811530E4930708F0BDC0883E910528F5E6
:1028C000803E910508F09DC0883A910588F4853ACC
:1028D000910508F08FC08130910509F492C00097EE
:1028E00009F48FC0049708F08CC0D0E0C0E089C024
:1028F0008F3B910508F489C0805C9109C03CD105EB
:10290000A0F30E944614EC017CC08115904250F463
:10291000C11581E0D80708F074C0C03FD10528F385
:10292000D0656FC0C11590E3D90708F079C0CE011A
:102930009F70E7CF811525E5920758F5811534E59D
:10294000930708F0A6C0811542E5940750F4C1151D
:1029500081E5D80708F471C0DC2FCC27C16FD06A9D
:1029600050C0982F969596959E0123703327C115D8
:10297000D34508F07FC0C1E0D0E002C0CC0FDD1F1E
:102980002A95E2F720E2929FC0011124C82BD92B8F
:102990006FC0C11589E5D807A8F4C11598E5D90716
:1029A00008F07CC0C11526E5D20708F09ECF8C2F19
:1029B0000E94FC15C82FD0E0DC2FCC27CC27DF717C
:1029C000D0621FC0C1153AE5D30708F46CC0CE0130
:1029D00090568115904208F088CF8D2F8F710E94FC
:1029E000FC1590E0982F882788279F719C012C2B3D
:1029F000E901E6CFC55AD0E0CC58DE4FC881D0E01F
:102A0000D064CE01DF91CF910895C85AD0E0CC0FA9
:102A1000DD1FCA5BDE4F0990D881C02DD464F1CF91
:102A2000CE019927D3FF03C0EC01D86CEACFEC01AB
:102A3000D06CE7CFDF70D06AE4CFCE01E4E09695AA
:102A40008795EA95E1F783702C2F269526952370BC
:102A500090E2299F90011124382B8C2F8370C1E0C4
:102A6000D0E002C0CC0FDD1F8A95E2F7C22BD32B3A
:102A7000DC68C7CFC1E0D0E002C0CC0FDD1F2A95D3
:102A8000E2F730E2939FC0011124C82BD92BDA68FA
:102A9000B8CFD82FCC27C46FD06AB3CFDC2FCC27C8
:102AA000C06FD06AAECF8C2F8F700E94FC1534E0BF
:102AB000D695C7953A95E1F7CF709C2FEC01D06978
:102AC000A0CF0E94961C0C944E1482389105B1F14F
:102AD000B0F48133910509F475C048F48932910549
:102AE00009F469C08A32910509F473C008958533E9
:102AF000910509F459C08933910501F10895833E88
:102B00009105A9F138F4803E9105F9F0823E9105D6
:102B100049F10895863E9105A9F1873E9105C9F1D5
:102B2000843E910519F52091830221FF1FC08091F9
:102B3000820284FD14C087EE90E008952091820205
:102B40002370A1F080EE90E008952091820220FD94
:102B500047C03091830230FF09C024FF44C090E099
:102B600080E004C02091820222FDF7CF08952091D9
:102B7000820222FD3BC03091830230FDE3CF24FF6F
:102B8000F5CFEDCF2091820223FFF0CF24FDE7CFD8
:102B9000D2CF2091820223FD2CC03091830231FFDD
:102BA000EECF84EE90E008952091820225FFDECFE3
:102BB00089E290E008952091820225FFD7CF85E336
:102BC00090E008952091820226FFD0CF8AE290E023
:102BD00008952091820226FFC9CF81E390E00895F5
:102BE00089E390E0089583EE90E0089582EE90E00E
:102BF000089586EE90E008959091820292FF06C0BB
:102C0000282F28712830F9F4877F846093FF06C04D
:102C1000282F28712831F1F4877E84612091830266
:102C200020FF06C0382F38713830D9F4877F816093
:102C300021FF06C0282F28712831D1F4877E8161B9
:102C400094FD877E0895282F24712430F9F68B7F18
:102C50008860DCCF282F2471243101F78B7E8861B6
:102C6000DDCF382F3171313019F78E7F8860E0CF9A
:102C7000282F2171213121F78E7E8861E1CF80E0FC
:102C800008950C947D120E9469172FEF86E791E05A
:102C9000215080409040E1F700C000000E94691779
:102CA00080E00E947A1660FF04C00E9441160C94D6
:102CB0005E2108950C9443160E948312811102C074
:102CC0000E9427130E948E12809341020E94961246
:102CD00090938302809382020E945A160E9492125D
:102CE0000E943D0D8091C5010C94500D0C94750708
:102CF0000C94760794E0899FF0011124E856FD4F6B
:102D000060817181828193810895089580EA8A9516
:102D1000F1F7089500C008950C948616F894E82FF2
:102D2000E295EF70F0E031A1282F2F7081E090E064
:102D300001C0880F2A95EAF7982F9095932391A3C5
:102D400092A1892B82A378940895CF93DF93C9E849
:102D5000D1E089918F3F11F00E948E1681E0CE382C
:102D6000D807B9F7C7E7D1E089918F3F11F00E94EA
:102D70008E1681E0C938D807B9F7DF91CF91089551
:102D80004F925F926F927F928F929F92AF92BF927B
:102D9000DF92EF92FF920F931F93CF93DF938C01FB
:102DA000D62EC62FD0E0CE0187579E4F7C01FC0166
:102DB00020812F3F09F462C0F894E22FE295EF7072
:102DC000F0E031A12F7081E090E001C0880F2A95DA
:102DD000EAF7932F982B91A392A18095892382A340
:102DE00078940E948A16E7E7F1E030E020E0812C39
:102DF000912C5401412C512C3201439481918F3FED
:102E000009F44CC0A82FA295AF70B0E090964C91F9
:102E100050E08F7002C0559547958A95E2F740FDC6
:102E20003DC0D301C201022E04C0880F991FAA1F02
:102E3000BB1F0A94D2F7882A992AAA2ABB2A2F5F95
:102E40003F4F22313105D1F6F70180818F3F11F0DC
:102E50000E948E1661E081149104A104B10409F46A
:102E600060E08D2D0E948C16CC0FDD1FCC0FDD1F76
:102E7000C00FD11F88829982AA82BB82DF91CF9135
:102E80001F910F91FF90EF90DF90BF90AF909F90B8
:102E90008F907F906F905F904F90089580E090E0CA
:102EA000DC01C9CF0E94A516E4E8F2E0A8E9B2E08F
:102EB00011921192119211921D921D921D921D92CA
:102EC00082E0E839F807A1F785E00E94B4170C9476
:102ED000FC07FF920F931F93CF93DF93CDB7DEB71D
:102EE00064970FB6F894DEBF0FBECDBF8E010F5FA3
:102EF0001F4F84E1F80111928A95E9F7F12C6F2DAB
:102F0000C8010E94C016F394F5E0FF12F8CF44E127
:102F100050E0B80184E892E00E942B29FF24F3944A
:102F2000009709F4F12C892B41F084E1F801A4E821
:102F3000B2E001900D928A95E1F72F2D45E068E906
:102F400072E084E892E00E94B5170E9402088F2D7B
:102F500064960FB6F894DEBF0FBECDBFDF91CF9160
:102F60001F910F91FF9008950895FF920F931F9363
:102F7000CF93DF93F82ED92F8B01C42F222349F052
:102F800081E0809344020E94132190934302809336
:102F9000420280914402882399F0809142029091EC
:102FA00043020E942B21059758F0EF2DFD2FD801E9
:102FB00090E080E0D0E08C179D0744F0109244022E
:102FC000DF91CF911F910F91FF9008950191119181
:102FD000219131910D931D932D933D930196EBCF4C
:102FE0000E948D200E9428230E9441230E94532387
:102FF0000E945F13FBCF80914B0280FF12C0609153
:10300000070185E0689FB001112475956795759556
:10301000679560387105A8F561157105A1F1862FD6
:10302000089581FF09C06091070185E0689FB001A4
:10303000112475956795EDCF6091070182FD0AC057
:1030400080914A028823D1F0909106016091070196
:10305000891728F085E0689FB0011124DACF869F98
:10306000B001112485E0869F9001879F300D1124C7
:10307000692F70E0C9010E94F628CBCF65E070E0AF
:10308000CECF8FE7089581E0089580914B0280FFB5
:103090000CC06091030170E0759567957595679513
:1030A0006115710549F1862F089581FF06C0609171
:1030B000030170E075956795F3CF6091030182FD80
:1030C0000BC0909149029923A1F060910201809177
:1030D0000301961738F0682F70E06038710500F32F
:1030E0008FE70895899FC001112470E00E94F6289F
:1030F000F4CF61E070E0D7CF81E00895803F31F4F4
:103100000E94FB17819580934F020895813F19F427
:103110000E94FB17F8CF823F31F40E94FB17819584
:1031200080934E020895833F19F40E94FB17F8CF55
:10313000893F29F40E9445188093500208958A3FE0
:1031400021F40E9445188195F7CF8B3F31F40E94FE
:10315000451881958093510208958C3F19F40E947F
:103160004518F8CF9CE0980F953070F4845F990B68
:1031700021E030E001C0220F8A95EAF780914D02EC
:10318000822B80934D0208958D3F31F480914B0244
:10319000816080934B0208958E3F21F480914B0211
:1031A0008260F7CF8F3FB9F780914B028460F1CFF7
:1031B00040914E02803F59F480914F0287FF0DC02D
:1031C00010924F0241110BC010924A0208C0813F79
:1031D00081F480914F0218169CF3442381F0809172
:1031E000500290915102892B09F05AC01092490265
:1031F0000895823F49F447FFF0CF10924E0280912C
:103200004F028111ECCFE0CF833F19F41416ACF3D9
:10321000E4CF90915002893F29F41916F4F61092E8
:103220005002DBCF8A3F19F497FFD7CFF8CF9091A8
:1032300051028B3F29F497FFD0CF10925102CDCF8E
:103240008C3F19F41916CCF3C8CF9CE0980F953039
:1032500090F4845F990B21E030E0B90102C0660F61
:10326000771F8A95E2F7CB01809590914D028923D3
:1032700080934D02B2CF8D3F31F480914B028E7F0F
:1032800080934B02AACF8E3F21F480914B028D7F19
:10329000F7CF8F3F09F0A1CF80914B028B7FF0CF0A
:1032A00008950E9413219C0190914E0280914F023B
:1032B000982B21F0309348022093470290915002BE
:1032C00080915102982B21F03093460220934502C1
:1032D0008CE492E00C94971FEF92FF920F931F9350
:1032E000CF93DF9300D000D000D0CDB7DEB786E01B
:1032F000ECE4F2E0DE01119601900D928A95E1F77F
:10330000E0904E02F0904F02009150021091510255
:1033100010924E0210924F021092500210925102DF
:103320008E2D8F2991F080914702909148020E9442
:103330002B21AC0190914A02992309F43FC080915E
:1033400008018417150608F447C0802F812B91F0DF
:1033500080914502909146020E942B21AC019091F0
:103360004902992309F477C0809104018417150656
:1033700008F47FC080914E0290914F02892B90916A
:103380005002892B90915102892B11F00E94511902
:1033900086E0FE013196ACE4B2E001900D928A9590
:1033A000E1F726960FB6F894DEBF0FBECDBFDF91D2
:1033B000CF911F910F91FF90EF90089520910901F7
:1033C0008AE0289F900111242417350708F0BDCF0B
:1033D0009F5F90934A0202C09F3FD1F7EE2059F0C1
:1033E0000E94FB179FEF1E140CF491E0899F802D23
:1033F000112480934E02FF2059F00E94FB179FEF8B
:103400001F140CF491E0899F802D112480934F02AA
:1034100030914E02332309F498CF20914F0222239A
:1034200009F493CF45EB3403C0011124992359F0DB
:1034300090934E0245EB240390011124332339F07D
:1034400030934F0282CF81E080934E02F3CF81E030
:1034500080934F027ACF209105018AE0289F900146
:1034600011242417350708F085CF9F5F90934902F8
:1034700002C09F3FD1F7002359F00E9445189FEFEB
:1034800010160CF491E0899F802D11248093500236
:10349000112359F00E9445189FEF11160CF491E08A
:1034A000899F802D11248093510230915002332343
:1034B00009F460CF20915102222309F45BCF45EB40
:1034C0003403C0011124992359F09093500245EB25
:1034D000240390011124332339F0309351024ACF51
:1034E00081E080935002F3CF81E08093510242CF7C
:1034F00086E0ECE4F2E0DF011D928A95E9F7109294
:103500004A021092490210924B02089583E290E021
:103510000E943829813289F484E290E00E9438299F
:10352000823159F485E290E00E94382991E081309F
:1035300009F090E0892F8170089580E0FCCFCF934F
:10354000C82F6FEF811161E283E290E00E9446296B
:103550006FEFC11162E184E290E00E9446296FEFB3
:10356000C11161E085E290E0CF910C944629089565
:1035700086E290E00E943829682F70E090E080E0B9
:10358000089586E290E00C94462980E00E949F1AFC
:1035900060E070E0CB010E94C11A0E940E1C0E94E4
:1035A000FA1C81E00C949F1A0E94B71A0E94861A96
:1035B000811102C00C94C51A0895CF93FB01C281FA
:1035C000CC2309F19C0122513F452031310520F5E2
:1035D00082510E940A1DC0E08C2FCF91089581E096
:1035E0000E94630D43E062E081E00E94F307F3CFA5
:1035F00081E00E946E0D43E062E081E00E94F307EB
:10360000EBCF82E0F6CF8031FFE59F0789F3813170
:103610009F45B9F3C1E0E0CF8031EFE59E07F9F2B5
:1036200081319F45C9F682E0DBCF2FEFFC0120837B
:103630000895EF92FF920F931F93CF93DF93EC01C6
:10364000E62EE881E150E33108F05FC0F0E0E65695
:10365000F64D0C940A29198289E08A836E2DCE01D9
:10366000DF91CF911F910F91FF90EF900C941D224D
:103670008981823069F0833071F08130E1F40E94F9
:103680001F210E9410296A837B838C839D83E6CF50
:103690000E94B81AF6CF8E01F12C8F2D0E947A1657
:1036A000F801828373836483F3940D5F1F4FF5E009
:1036B000FF12F3CFD3CF6E2DCE010E94151BCECFBC
:1036C00089818230C1F76A817B818C819D810E94D2
:1036D00010290E94C11AC2CF4B816A8189810E9440
:1036E000E01B9827892798279D838C83B7CF2C814F
:1036F0003D813227232732274B816A8189810E94AD
:10370000F91BACCF0E940E1CA9CF8FEF8883A6CFE8
:103710000E94A31C8983A2CF0E94A51C98278927F9
:1037200098279A8389839ACF6B8170E089819A81E7
:10373000AE014C5F5F4F9827892798270E94A81CED
:103740008DCF6B8170E089819A81AE014C5F5F4FB4
:103750009827892798270E94CF1C80CF0E94FA1CA7
:103760007DCF0E94CE1BD6CF6B8170E089819A817C
:10377000AE014C5F5F4F9827892798270E94461C0F
:103780006DCF6B8170E089819A81AE014C5F5F4F94
:103790009827892798270E946C1C60CF84E00895A1
:1037A00050E0440F551F94E2699F400D511D1124B4
:1037B00094EB899F400D511D1124CA0187960895ED
:1037C0000F931F93CF93DF930E94D01B8C010E9415
:1037D0003829C82FD0E0DC2FCC27C80101960E94E1
:1037E00038299E01282BC901DF91CF911F910F919C
:1037F00008950F931F93CF93DF93122F032F0E94EF
:10380000D01BEC01602F0E944629612FCE0101964A
:10381000DF91CF911F910F910C944629AF92BF92E7
:10382000CF92DF92EF92FF921F93CF93DF938CEAB8
:10383000C82E80E0D82ED0E07601C0E014C0F5019B
:1038400025913491412F6C2F8D2F0E94F91B82E01E
:10385000A80EB11C1F5F123191F784E2E80EF11C33
:10386000CF5FC53019F0570110E0E9CFDF5F84EB7F
:10387000C80ED11CD43001F7DF91CF911F91FF907A
:10388000EF90DF90CF90BF90AF900895EF92FF92AE
:103890000F931F93CF93DF93EC018A017C01E60E17
:1038A000F71ECE018796CE15DF0539F4DF91CF9153
:1038B0001F910F91FF90EF900895C03D22E0D20735
:1038C00040F40E943829F80180830F5F1F4F219632
:1038D000E8CFF8011082F9CFCF92DF92EF92FF92FA
:1038E0000F931F93CF93DF937C016A018C01060F26
:1038F000171FEC01CE018796C017D10749F4DF915D
:10390000CF911F910F91FF90EF90DF90CF9008958E
:10391000C03D22E0D20740F4FE01EE19FF09EC0D94
:10392000FD1D60810E9446292196E4CF462F8430F8
:1039300038F4753028F4623118F4672F0C94E01BCA
:1039400090E080E0089580E1089589E091E0089595
:10395000EF92FF920F931F93CF93DF93EC018A01B5
:103960007C01E60EF71ECE0189509D4FCE15DF0576
:1039700039F4DF91CF911F910F91FF90EF9008954F
:10398000C93021E0D20740F40E943829F801808331
:103990000F5F1F4F2196E7CFF8011082F9CFCF922A
:1039A000DF92EF92FF920F931F93CF93DF937C01EF
:1039B0006A018C01060F171FEC01CE0189509D4F43
:1039C000C017D10749F4DF91CF911F910F91FF905C
:1039D000EF90DF90CF900895C93021E0D20740F4F6
:1039E000FE01EE19FF09EC0DFD1D60810E944629C4
:1039F0002196E3CFCF93DF93C7EFD2E060E0CE0113
:103A00000E9446292196C11584E0D807B9F7DF91B5
:103A1000CF910895DF92EF92FF920F931F93CF9370
:103A2000DF9300D000D0CDB7DEB7F82E8FE08F1532
:103A300040F08FEF93E00E94382907EF12E08823CF
:103A4000C1F00F900F900F900F90DF91CF911F91C9
:103A50000F91FF90EF90DF900895011584E0180713
:103A600081F3C8010E943829811101C0FA940F5FC7
:103A70001F4FF110F2CF19821A821B821C82DD24A3
:103A8000D39478018FEFE81AF80AC8010E94382908
:103A900089831A828823A9F29FEF980F933078F4D4
:103AA0008A83D9820E5F1F4FC7010E9438298B83FA
:103AB000882339F2CE0101960E943A09E2CF8701AC
:103AC000F9CF0F931F93CF93DF93C42FD22FFC0115
:103AD00082818823C9F0409354020E94132190935D
:103AE00053028093520280E28C0F883008F050C05D
:103AF000C77081E001C0880FCA95EAF7DF91CF91C6
:103B00001F910F910C94960A10915402141335C012
:103B100080915202909153020E942B21883C910582
:103B200060F5C0E2CD0F1D17B9F080E2810F88303B
:103B300040F4177081E001C0880F1A95EAF70E94DF
:103B40009D0AC83048F481E09D2F977001C0880F0E
:103B50009A95EAF70E94960A802F0E948E0AC83032
:103B6000B8F4D77081E001C0880FDA95EAF7DF91E9
:103B7000CF911F910F910C949D0A80E28C0F883099
:103B800038F4C77081E001C0880FCA95EAF7EFCF1B
:103B9000DF91CF911F910F9108950F939C01CB015D
:103BA000233F4CE5340759F1A8F4283DFCE53F07D5
:103BB00001F1293D4CE53407D1F1273D3C4591F415
:103BC00006E221EE41EE67ED7CE50E94611D80E09A
:103BD0000F910895253FFCE53F07E9F0B0F0263F3F
:103BE0003C45F9F0FC018281882339F1109254029E
:103BF000EFCF07E225EE45EE68ED7CE5E6CF06E285
:103C000021EE40EE63EF7CE5E0CF07E225EE44EEE7
:103C100064EF7CE5DACF06E221EE42EE65EF7CE56B
:103C2000D4CF07E225EE46EE66EF7CE5CECF08E284
:103C300021E045EE69ED7CE5C8CF81E0C9CFCF93A7
:103C4000DF93EC01FB018281882309F419C1C230A2
:103C5000FCE5DF07C0F1C6319CE5D90730F09E01D5
:103C60002A5F3C452930310570F50E9496129093E9
:103C7000830280938202C031ECE5DE0709F4CFC0F5
:103C800008F05BC0C8308CE5D80709F4B6C088F5E9
:103C9000C430ECE5DE0709F4A8C0C0F4C2308CE5FE
:103CA000D80709F49CC0809182028260C330DC4551
:103CB00009F498C080918202909183020E94A4121C
:103CC0000E94EA0C80E0DF91CF91089580918202FA
:103CD0008061C630ECE5DE0709F484C08091820281
:103CE0008860C730DC4508F47DC080918202806224
:103CF00079C0CC308CE5D80709F489C070F4809184
:103D000082028C60CA30ECE5DE0709F46BC008F46F
:103D100078C0809182028E7F65C0CE308CE5D80756
:103D200009F479C0809182028B7FCF30DC4508F4A2
:103D300059C0809182028F7E55C0CB3FECE5DE07F3
:103D400009F457C030F5C3318CE5D80709F46FC0CA
:103D500078F4C131ECE5DE0709F465C0C231DC4519
:103D600009F0A8CF0E94EA0C809182028F773AC0B6
:103D7000C5318CE5D80709F462C008F476C080919B
:103D800083028160CA3FDC4509F094CF80938302AF
:103D900091CFCF3FFCE5DF0709F44DC088F4809157
:103DA00083028D7FCD3F9CE5D90781F3809183020B
:103DB0008E7FCE3FDC4550F3809183028360E6CF57
:103DC000C130FDE5DF0709F459C008F444C080E0C4
:103DD000C230DD4509F06ECF0E9429136BCF809170
:103DE000820281608093820265CF8091820284602A
:103DF000F9CF809183028260C9CF80918202806472
:103E0000F1CF0E94EA0C809182028068EBCF809112
:103E100082028D7FE7CF80918202877FE3CF8091FE
:103E200082028F7DDFCF809182028F7BDBCF8091FA
:103E30008202837FD7CF809183028C7FA7CF80912E
:103E4000820282FB992790F921E0922790FB82F968
:103E500090FB83F9C7CF80918302982F9095917042
:103E60008E7F892B90FB81F991CF0E94EA0C909173
:103E70008202892F97FB87F98058B4CF81E0ACCFBD
:103E800081E021CFCF93DF93EB0186319C4511F583
:103E90000E94C0119A81992399F08A7A91E009F4DD
:103EA00090E090935502811109C089E20E947A1135
:103EB0000E94101280E0DF91CF91089585E3F6CF44
:103EC00080915502811104C089E20E948111F0CFD6
:103ED00085E3FBCF81E0EFCF90935B0280935A02A2
:103EE0000895E0915A02F0915B02309721F0019021
:103EF000F081E02D099480E00895E0915A02F0915C
:103F00005B02309799F020911401222359F02091FF
:103F1000820227FF07C0DC012C9111962C93119788
:103F200025E02C930280F381E02D09940895E0911F
:103F30005A02F0915B02309739F022E0DC012C93B9
:103F40000480F581E02D0994089520915802309164
:103F500059022817390771F090935902809358023B
:103F6000E0915A02F0915B02309721F00680F781D0
:103F7000E02D099408952091560230915702281798
:103F8000390771F09093570280935602E0915A02DC
:103F9000F0915B02309721F00084F185E02D0994C7
:103FA0000895FC01329680911401882321F08091BC
:103FB00082029EE187FF96E080E0915008F4089528
:103FC00021912223D1F38F5FF8CF662301F1209155
:103FD00014012223F1F02091820227FF1AC0462FFC
:103FE0004695469546954E3190F4677021E030E055
:103FF00002C0220F331F6A95E2F7840F911DFC0166
:10400000828190E02823392381E0232B69F480E02A
:104010000895FC01329608962191261721F0E817A1
:10402000F907D1F7F4CF81E008959C01FC013296A5
:104030009FEF80E04191461751F09F3F19F44111E5
:1040400001C0982F8F5F8630A9F79F3F09F408952C
:10405000290F311D97FD3A95F90162830895FC01FE
:10406000329608962191261303C0DF0111971C9206
:10407000E817F907B9F70895E62FE695E695E6956E
:10408000EE3168F4E80FF92FF11D677021E030E0A0
:1040900001C0220F6A95EAF78281822B82830895FC
:1040A000E62FE695E695E695EE3170F4E80FF92FE8
:1040B000F11D677021E030E001C0220F6A95EAF738
:1040C00020958281282322830895209114012223A0
:1040D00029F02091820227FD0C943C200C9415209D
:1040E00020911401222329F02091820227FD0C94B3
:1040F00050200C942F20FC013296809114018823CB
:1041000051F08091820287FF06C08EE1DF011D928F
:104110008A95E9F7089586E0F9CF089508950895FE
:104120000C948F208091B402843049F10E94902039
:1041300080E00E94440910925C0288E190E020E453
:104140000FB6F894A895809360000FBE209360008E
:1041500083B7817F846083BF83B7816083BF789496
:10416000889583B78E7F83BF0FB6F894A89580910A
:104170006000886180936000109260000FBE089517
:104180000895CF930E948E200E9469170E94C0203C
:10419000C0E08C2F0E947A16672B682B692B31F4B4
:1041A000CF5FC530B1F780E0CF91089581E0FCCFBB
:1041B00008950C94D8200E94EA0C0E94711F0E945E
:1041C00044090C94D9201F921FB61F9211248F937B
:1041D0009F93AF93BF9380915C02811113C0809134
:1041E000AC029091AD02A091AE02B091AF024196A7
:1041F000A11DB11D8093AC029093AD02A093AE02BD
:10420000B093AF02BF91AF919F918F911F901FBE4E
:104210001F90189582E084BD93E095BD9AEF97BDFD
:1042200080936E0008952FB7F8948091AC0290911E
:10423000AD02A091AE02B091AF022FBF08952FB78B
:10424000F8946091AC027091AD028091AE029091B1
:10425000AF022FBF08959C014FB7F8948091AC0234
:104260009091AD02A091AE02B091AF024FBF821B00
:10427000930B089578941F921FB61F9211248F9369
:104280009F93AF93BF938091AC029091AD02A091A8
:10429000AE02B091AF020196A11DB11D8093AC0298
:1042A0009093AD02A093AE02B093AF02BF91AF91D5
:1042B0009F918F911F901FBE1F90189581E0809352
:1042C000E00080E28093D8001092C9008FE19EE464
:1042D0000197F1F700C0000087E090EBDC018093CC
:1042E000BD029093BE02A093BF02B093C00288E1CA
:1042F0009CE00FB6F894A895809360000FBE909351
:104300006000FFCF90939F0180939E01089580915C
:10431000800208959091B402943029F580935D0253
:1043200070935F0260935E029093E9008FEF90912B
:10433000E800815095FD06C095ED9A95F1F70000D3
:104340008111F5CF8091E80085FF0DC050E040E07D
:1043500063E070E08DE592E00E9416248091E80011
:104360008E778093E8000895BC0184E00C948A2144
:10437000BC0183E00C948A219C0184E08093E900D5
:104380009FEF8091E800915085FD06C085ED8A95EC
:10439000F1F700009111F5CF8091E80085FF0CC086
:1043A00050E040E066E070E0C9010E941624809170
:1043B000E8008E778093E8000895CF93DF93EC01B7
:1043C000809114018823B1F18091820287FF32C06D
:1043D00060E284E08093E9008FEF9091E8008150E3
:1043E00095FD06C095ED9A95F1F700008111F5CF86
:1043F0008091E80085FF1BC08091140170E050E0BF
:1044000040E0811104C050E040E068E070E0CE017F
:104410000E9416248091E8008E778093E80080E265
:10442000FE01A0E6B2E001900D928A95E1F7DF91DE
:10443000CF91089568E081E0CDCFCF93FC01603249
:1044400021F58091B402843001F5C091E900CF706C
:104450002091EC00922F917020FD90E8C92B82E012
:104460008093E9008091E80080FF0CC050E040E0BC
:1044700060E270E0CF010E9416248091E8008E7700
:104480008093E800CF70C093E900CF9108958091A8
:10449000B302811109C00E94F5250E945226809125
:1044A000E20084608093E20008951092B3020895C0
:1044B00008950895089542E061EC81E00E9471251D
:1044C00042E261EC84E00E94712542E261EC82E00C
:1044D0000E94712542E260EC83E00C94712580918A
:1044E000B602833009F461C030F48130D1F18230FA
:1044F00009F49DC008958A3009F489C08B3009F40D
:104500006FC0893009F050C08091B502813209F046
:104510004BC08091B9029091BA02009719F00297AE
:1045200009F042C08091E800877F8093E800809185
:10453000E80082FF35C09091F3008091F20002976D
:1045400029F48091F1008B7F813021F48091F1007A
:10455000809380028091E8008B778093E8000C9430
:10456000A5258091B502813AF9F48091E800877F12
:104570008093E8008091B9029091BA02892B61F48E
:1045800060E280E692E070E00E94B4248091E8004E
:104590008B778093E800089560E090E080E0F3CFAF
:1045A0008091B4028111C3CF08958091B502813A00
:1045B000D9F78091B9029091BA02892BA9F780911D
:1045C000E800877F8093E8008091E80080FFFCCFBF
:1045D000809114018093F1008091E8008E77BDCF27
:1045E0008091B502813201F78091B9029091BA02AF
:1045F000892BD1F68091E800877F8093E8000E94A4
:10460000A5258091B702809314010C94EA0C809147
:10461000B502813249F68091E800877F8093E800F7
:104620000E94A5258091B80280938102089580910F
:10463000B502813A09F0B8CF8091E800877F809376
:10464000E8008091E80080FFFCCF80918102C2CF1A
:1046500084B7877F84BF0FB6F894A89580916000D7
:10466000886180936000109260000FBE80E890E047
:104670000FB6F89480936100909361000FBE0C9484
:104680004F130E94F5250E945226E2EEF0E0808151
:104690008460808378940E94DB280E9463138AE000
:1046A00091E00C946C1FCF93DF93CDB7DEB7A0974A
:1046B0000FB6F894DEBF0FBECDBF8091B402853037
:1046C00031F48091B402853091F10E94DB200E9488
:1046D0006B138091B402843009F583E08093E90084
:1046E0008091E80082FF1AC08091E80090E085FF89
:1046F00009C050E040E060E270E0CE0101960E9407
:10470000652491E08091E8008B778093E8009923FD
:1047100029F060E2CE0101960E94191BA0960FB607
:10472000F894DEBF0FBECDBFDF91CF9108950E94F8
:1047300092208091B202882321F20E94C120882316
:1047400009F4BFCF0E9400240E94EA0CBACF0C9457
:10475000A923292F33272330310521F168F4213093
:10476000310509F443C02230310509F444C090E01A
:1047700080E030E020E026C02132310551F12232C4
:104780003105A9F76330710590F7FB01EE0FFF1FAC
:10479000EF56FE4F2081318162577E4FFB018081B1
:1047A00090E010C099278130910581F0009729F0A1
:1047B0000297E9F6ECE9FCE002C0E8ECFCE0849149
:1047C00090E09F01FA01318320830895E0EBFCE043
:1047D000F6CF6330710558F6660F771FFB01E95677
:1047E000FE4F2081318189E090E0ECCF82E190E0C2
:1047F00027E23DE0E7CF8BE590E02CEC3CE0E2CF18
:1048000080E189BD82E189BD09B400FEFDCF8091C0
:10481000D8008F7D8093D8008091E00082608093E3
:10482000E0008091E00081FDFCCF0895AF92BF923F
:10483000CF92DF92FF920F931F93CF93DF936C0180
:10484000EB018A010E94C425F82E811123C00115B5
:10485000110539F0F80180819181C81BD90BC80E70
:10486000D91EB12CA12C2097A9F08091E80085FDDC
:1048700022C08091E8008E778093E8000115110531
:10488000A1F0F80180819181A80EB91EB182A082A9
:1048900085E0F82E8F2DDF91CF911F910F91FF9022
:1048A000DF90CF90BF90AF9008950E94C4258823D9
:1048B000D1F2F82EEFCFF60181916F018093F100D4
:1048C0002197FFEFAF1ABF0ACECFAF92BF92CF9220
:1048D000DF92FF920F931F93CF93DF936C01EB0155
:1048E0008A010E94C425F82E811123C001151105EB
:1048F00039F0F80180819181C81BD90BC80ED91EEF
:10490000B12CA12C2097A9F08091E80085FD22C050
:104910008091E8008B778093E80001151105A1F0E4
:10492000F80180819181A80EB91EB182A08285E034
:10493000F82E8F2DDF91CF911F910F91FF90DF9077
:10494000CF90BF90AF9008950E94C4258823D1F2E4
:10495000F82EEFCF8091F100F60181936F0121973E
:10496000FFEFAF1ABF0ACECFFC018091BB0290913E
:10497000BC0286179707A0F06115710529F4909184
:10498000E8009E779093E80090E06115710551F47E
:10499000911108C08091E80082FF34C080E0089542
:1049A000BC01F2CF8091B4028823C1F18530C1F1FE
:1049B0008091E80083FD30C08091E80082FDEACF5D
:1049C0008091E80080FFE1CF8091F3002091F20018
:1049D000382F6115710519F02830310558F091E034
:1049E0002830310509F090E02091E8002E772093DF
:1049F000E800CBCF81918093F100615071092F5F66
:104A00003F4FE7CF8091B402882341F0853041F0D9
:104A10008091E80083FFBECF81E0089582E0089591
:104A200083E00895FC018091BB029091BC0286173F
:104A30009707A0F06115710529F48091E8008E7741
:104A40008093E80090E06115710551F4911108C060
:104A50008091E80082FF35C080E00895BC01F2CF6C
:104A60008091B4028823C9F18530C9F18091E800B2
:104A700083FD31C08091E80082FDEACF8091E8009B
:104A800080FFE1CF8091F3002091F200382F611573
:104A9000710519F02830310558F091E028303105C2
:104AA00009F090E08091E8008E778093E800CBCF0A
:104AB00084918093F1003196615071092F5F3F4FCF
:104AC000E6CF8091B402882341F0853041F0809197
:104AD000E80083FFBDCF81E0089582E0089583E080
:104AE0000895982F973028F08F708093E90081E027
:104AF00008959093E900242F762F50E0981731F015
:104B00007091EC002091ED005091F00021FD02C069
:104B10009F5FE8CF3091EB003E7F3093EB00309108
:104B2000ED003D7F3093ED003091EB00316030932C
:104B3000EB007093EC002093ED005093F000209177
:104B4000EE0027FDE5CF80E008958091B50287FF54
:104B500013C08091E80082FF06C08091E8008B7747
:104B60008093E80004C08091B4028111F2CF0895CF
:104B70008091B4028823D9F38091E80080FFF8CFB8
:104B80008091E8008E77ECCF2091E4003091E50031
:104B900095E6A9012091EC00822F817020FF06C0CC
:104BA0008091E80080FF06C080E008952091E80031
:104BB00022FD1AC08091B402882389F0853089F0E3
:104BC0008091EB0085FD0FC02091E4003091E5005D
:104BD00042175307F9F29150E1F684E0089582E01C
:104BE000089583E0089581E008950E9463260E945D
:104BF0006B26E0EEF0E0808181608083E8EDF0E0FC
:104C000080818F77808319BCA7EDB0E08C918E7F77
:104C10008C9380818F7E80831092B30208950F93CE
:104C20001F93CF93DF930E9463260E946B26C8EDEB
:104C3000D0E088818F7788838881806888838881A5
:104C40008F7D888319BC1092B4021092B00210922A
:104C5000B2021092B10200EE10E0F80180818B7F69
:104C6000808388818160888342E060E080E00E94E8
:104C70007125E1EEF0E080818E7F8083E2EEF0E04E
:104C8000808181608083808188608083F801808159
:104C90008E7F8083888180618883DF91CF911F918F
:104CA0000F910895E8EDF0E080818F7E8083E7ED3D
:104CB000F0E080818160808384E082BF81E0809326
:104CC000B3020C940F26E8EDF0E080818E7F8083A4
:104CD0001092E20008951092DA001092E100089517
:104CE0001F920F920FB60F9211242F933F934F9361
:104CF0005F936F937F938F939F93AF93BF93EF9344
:104D0000FF938091E10082FF0BC08091E20082FF5F
:104D100007C08091E1008B7F8093E1000E94DA2838
:104D20008091DA0080FF19C08091D80080FF15C003
:104D30008091DA008E7F8093DA008091D90080FF25
:104D400096C080E189BD82E189BD09B400FEFDCF36
:104D500081E08093B4020E9447228091E10080FFAD
:104D600019C08091E20080FF15C08091E2008E7F23
:104D70008093E2008091E20080618093E200809164
:104D8000D80080628093D80019BC85E08093B4027B
:104D90000E9459228091E10084FF2BC08091E200A3
:104DA00084FF27C080E189BD82E189BD89B5982F44
:104DB000917080FFFBCF8091D8008F7D8093D800C9
:104DC0008091E1008F7E8093E1008091E2008F7EF0
:104DD0008093E2008091E20081608093E200809104
:104DE000B002882309F449C084E08093B4020E9491
:104DF0005A228091E10083FF29C08091E20083FF65
:104E000025C08091E100877F8093E10082E080935C
:104E1000B4021092B0028091E1008E7F8093E10095
:104E20008091E2008E7F8093E2008091E2008061B9
:104E30008093E20042E060E080E00E947125809172
:104E4000F00088608093F0000E945822FF91EF915B
:104E5000BF91AF919F918F917F916F915F914F9192
:104E60003F912F910F900FBE0F901F90189519BC76
:104E70001092B4020E94552270CF8091E30087FD0A
:104E800093E09093B402B3CF1F920F920FB60F929C
:104E900011242F933F934F935F936F937F938F933F
:104EA0009F93AF93BF93CF93DF93EF93FF93D091F3
:104EB000E900DF708091EC00C82FC17080FDC0E870
:104EC0001092E9008091F000877F8093F000789441
:104ED0000E9488271092E9008091F00088608093FA
:104EE000F000CD2BCF70C093E900FF91EF91DF91DF
:104EF000CF91BF91AF919F918F917F916F915F9172
:104F00004F913F912F910F900FBE0F901F901895CA
:104F10001F93CF93DF93CDB7DEB7AA970FB6F89460
:104F2000DEBF0FBECDBF85EB92E02091F100FC010A
:104F30002193CF01F2E08D3B9F07B9F70E946F22CA
:104F40008091E80083FF1EC18091B5029091B60266
:104F50009A3008F017C1E92FF0E0E355F64D0C94B4
:104F60000A29803899F0823809F00CC18091B90281
:104F70008F70873008F006C18093E9008091EB00C4
:104F800085FB882780F91092E90006C08091B10264
:104F90009091B202911182609091E800977F909376
:104FA000E8008093F1001092F1008091E8008E7784
:104FB000E5C0882309F4D3C0823009F0E3C08091B2
:104FC000B7028111D6C08091B9028F702FEF280FE0
:104FD000263008F0D7C08093E9002091EB0020FF35
:104FE000C8C0933031F48091EB0080628093EB0075
:104FF000C0C09091EB0090619093EB0021E030E015
:1050000001C0220F8A95EAF72093EA001092EA0085
:105010008091EB008860EACF8111B4C01091B70293
:105020001F778091E3008078812B8093E30080914B
:10503000E800877F8093E8000E94A5258091E80022
:1050400080FFFCCF8091E30080688093E30082E0E2
:10505000111183E08093B40295C08058823008F02B
:1050600091C08091B7029091B8028C3D23E09207E5
:10507000A1F583E08A838AE289834FB7F894DE0141
:10508000139620E03EE051E2E32FF0E0509357000A
:10509000E49120FF03C0E295EF703F5FEF708E2F29
:1050A00090E0EA30C0F0C7968D939D932F5F243136
:1050B00059F74FBF8091E800877F8093E8006AE24C
:1050C00070E0CE0101960E94B4248091E8008B77B5
:1050D0008093E80057C0C096E7CF6091B902709105
:1050E000BA02AE014F5F5F4F0E94A723BC01892B1C
:1050F00009F448C09091E800977F9093E800898177
:105100009A810E941225E1CF8038E1F58091E80074
:10511000877F8093E8008091B0028093F10045CFB3
:10512000811130C09091B702923060F58091E80013
:10513000877F8093E8009093B0020E94A52580911C
:10514000B002882311F084E005C08091E30087FD60
:10515000FACF81E08093B4020E945B2213C0809159
:10516000B702813079F481E0933009F080E08093D8
:10517000B2021092E9008091E800877F8093E800F6
:105180000E94A5258091E80083FF0AC08091E80075
:10519000877F8093E8008091EB0080628093EB0032
:1051A000AA960FB6F894DEBF0FBECDBFDF91CF91A8
:1051B0001F9108950895CF938091B4028823A1F0A0
:1051C000C091E900CF709091EC00892F817090FD23
:1051D00080E8C82B1092E9008091E80083FD0E94CE
:1051E0008827CF70C093E900CF91089597FB072ED1
:1051F00016F4009407D077FD09D00E94172907FC08
:1052000005D03EF4909581959F4F089570956195D6
:105210007F4F0895EE0FFF1F0590F491E02D099444
:105220006927962769277827872778270895AA1B53
:10523000BB1B51E107C0AA1FBB1FA617B70710F081
:10524000A61BB70B881F991F5A95A9F780959095B3
:10525000BC01CD010895FB01DC0104C08D910190DA
:10526000801921F441505040C8F7881B990B0895CC
:10527000F999FECF92BD81BDF89A992780B508951E
:10528000A8E1B0E042E050E00C946C29262FF99997
:10529000FECF92BD81BDF89A019700B4021639F095
:1052A0001FBA20BD0FB6F894FA9AF99A0FBE089566
:1052B0000396272F0E9447290E944629252F0E94E6
:1052C0004729242F0C9447290196272F0E9447290C
:1052D0000C944629DC01CB01FC01F999FECF06C0F4
:1052E000F2BDE1BDF89A319600B40D9241505040A4
:1052F000B8F70895F894FFCFD80AD80A300B300BCE
:10530000820B9E0B050B050BA90B100C1F0C1F0C21
:105310007B0C050B050B840CF90CF90C020D020D2E
:10532000040D020D020D020DF90CF90C090D020D10
:10533000020D090D2B1B381B601B6C1B771B821B7E
:10534000851B851B851B851B851B881B8C1B941B44
:10535000A11BAE1BB11BB41BC11BB127D927C2288F
:0E536000D927C2280C282D28C228842890287E
:10536E0001022808641E140A321E8721DD21BC2189
:10537E00B821B42101E200E900EA00B500B600B799
:10538E0000CD008301CC008A0192019401210223F9
:10539E000224022502260227022A02B300B4006F5D
:1053AE00007000818283E200E900EA00B500B600D9
:1053BE00B700CD008301CC008A0192019401210235
:1053CE00230224022502260227022A02B300B40079
:1053DE006F007000818283676636C6F69697343505
:1053EE00F737F4F59430313233F0F1929190402248
:0E53FE00B6110E390D5B0DDE0CF70C170D000D
:00000001FF
